:020000020000FC
:0400000014C051C017
:020008003AC0FC
:10002A00F8940FED0DBF06E007BB00E008BB01E046
:10003A0005BF00E40BBF0AB70ABF07EB0BBD0BE114
:10004A000ABD00E00DBD0CBD00E409BF00E000934D
:10005A0060007894009160000030E1F302E008BB90
:10006A0000E00DBD0CBD03E00EBD00916000003044
:10007A0089F3FBCF4FB74F93013041F400E000936F
:10008A00600006E008BB00E00EBD14C000E000936B
:10009A00600000E008BB00E00EBD0CC04FB74F93F4
:1000AA00829B04C002E00093600004C001E0009358
:0A00BA00600000C04F914FBF189581
:00000001FF
